 dt_socket

 Timestamp is ffffffff (Sun Feb  7 06:28:15 2106)

 Preferred load address is 10000000

 Start         Length     Name                   Class
 0001:00000000 00002ba0H .text$mn                CODE
 0002:00000000 00000138H .idata$5                DATA
 0002:00000138 00000004H .00cfg                  DATA
 0002:0000013c 00000004H .CRT$XCA                DATA
 0002:00000140 00000004H .CRT$XCZ                DATA
 0002:00000144 00000004H .CRT$XIA                DATA
 0002:00000148 00000004H .CRT$XIZ                DATA
 0002:0000014c 00000004H .CRT$XPA                DATA
 0002:00000150 00000004H .CRT$XPZ                DATA
 0002:00000154 00000004H .CRT$XTA                DATA
 0002:00000158 00000008H .CRT$XTZ                DATA
 0002:0000015c 00000000H .gfids$y                DATA
 0002:00000160 00000da8H .rdata                  DATA
 0002:00000f08 00000004H .rdata$sxdata           DATA
 0002:00000f0c 00000288H .rdata$zzzdbg           DATA
 0002:00001194 00000004H .rtc$IAA                DATA
 0002:00001198 00000004H .rtc$IZZ                DATA
 0002:0000119c 00000004H .rtc$TAA                DATA
 0002:000011a0 00000008H .rtc$TZZ                DATA
 0002:000011a8 00000088H .xdata$x                DATA
 0002:00001230 0000005cH .edata                  DATA
 0002:0000128c 000000a0H .idata$2                DATA
 0002:0000132c 00000014H .idata$3                DATA
 0002:00001340 00000138H .idata$4                DATA
 0002:00001478 00000418H .idata$6                DATA
 0003:00000000 00000038H .data                   DATA
 0003:00000038 000007bcH .bss                    DATA
 0004:00000000 00000060H .rsrc$01                DATA
 0004:00000060 00000328H .rsrc$02                DATA

  Address         Publics by Value              Rva+Base       Lib:Object

 0000:00000000       ___guard_fids_table        00000000     <absolute>
 0000:00000000       ___hybrid_code_map_count   00000000     <absolute>
 0000:00000000       ___guard_longjmp_table     00000000     <absolute>
 0000:00000000       ___hybrid_code_map         00000000     <absolute>
 0000:00000000       ___guard_fids_count        00000000     <absolute>
 0000:00000000       ___x64_code_ranges_to_entry_points 00000000     <absolute>
 0000:00000000       ___guard_iat_table         00000000     <absolute>
 0000:00000000       ___guard_eh_cont_count     00000000     <absolute>
 0000:00000000       ___arm64x_redirection_metadata 00000000     <absolute>
 0000:00000000       ___arm64x_extra_rfe_table_size 00000000     <absolute>
 0000:00000000       ___arm64x_extra_rfe_table  00000000     <absolute>
 0000:00000000       ___x64_code_ranges_to_entry_points_count 00000000     <absolute>
 0000:00000000       ___guard_iat_count         00000000     <absolute>
 0000:00000000       ___dynamic_value_reloc_table 00000000     <absolute>
 0000:00000000       ___guard_longjmp_count     00000000     <absolute>
 0000:00000000       ___arm64x_native_entrypoint 00000000     <absolute>
 0000:00000000       ___enclave_config          00000000     <absolute>
 0000:00000000       ___hybrid_auxiliary_iat    00000000     <absolute>
 0000:00000000       ___arm64x_redirection_metadata_count 00000000     <absolute>
 0000:00000000       ___AbsoluteZero            00000000     <absolute>
 0000:00000000       ___guard_eh_cont_table     00000000     <absolute>
 0000:00000000       ___volatile_metadata       00000000     <absolute>
 0000:00000001       ___safe_se_handler_count   00000001     <absolute>
 0000:00000100       ___guard_flags             00000100     <absolute>
 0000:00000000       ___ImageBase               10000000     <linker-defined>
 0001:00000000       ___local_stdio_printf_options 10001000 f i socketTransport.obj
 0001:00000006       __vfprintf_l               10001006 f i socketTransport.obj
 0001:0000002a       __vsnprintf_l              1000102a f i socketTransport.obj
 0001:00000178       _fprintf                   10001178 f i socketTransport.obj
 0001:0000044d       _jdwpTransport_OnLoad@16   1000144d f   socketTransport.obj
 0001:0000164f       _sprintf                   1000264f f i socketTransport.obj
 0001:000017bf       _DllMain@12                100027bf f   socket_md.obj
 0001:00001810       _dbgsysAccept              10002810 f   socket_md.obj
 0001:00001823       _dbgsysBind                10002823 f   socket_md.obj
 0001:00001836       _dbgsysConfigureBlocking   10002836 f   socket_md.obj
 0001:00001863       _dbgsysConnect             10002863 f   socket_md.obj
 0001:000018a2       _dbgsysCurrentTimeMillis   100028a2 f   socket_md.obj
 0001:0000193b       _dbgsysFinishConnect       1000293b f   socket_md.obj
 0001:000019d5       _dbgsysFreeAddrInfo        100029d5 f   socket_md.obj
 0001:000019e0       _dbgsysGetAddrInfo         100029e0 f   socket_md.obj
 0001:000019f7       _dbgsysGetLastIOError      100029f7 f   socket_md.obj
 0001:00001a37       _dbgsysGetSocketName       10002a37 f   socket_md.obj
 0001:00001a4a       _dbgsysHostToNetworkLong   10002a4a f   socket_md.obj
 0001:00001a55       _dbgsysHostToNetworkShort  10002a55 f   socket_md.obj
 0001:00001a60       _dbgsysListen              10002a60 f   socket_md.obj
 0001:00001a6f       _dbgsysNetworkToHostLong   10002a6f f   socket_md.obj
 0001:00001a7a       _dbgsysNetworkToHostShort  10002a7a f   socket_md.obj
 0001:00001a85       _dbgsysPoll                10002a85 f   socket_md.obj
 0001:00001b50       _dbgsysRecv                10002b50 f   socket_md.obj
 0001:00001b67       _dbgsysSend                10002b67 f   socket_md.obj
 0001:00001b7e       _dbgsysSetSocketOption     10002b7e f   socket_md.obj
 0001:00001c5b       _dbgsysSocket              10002c5b f   socket_md.obj
 0001:00001c84       _dbgsysSocketClose         10002c84 f   socket_md.obj
 0001:00001ccb       _dbgsysTlsAlloc            10002ccb f   socket_md.obj
 0001:00001cd1       _dbgsysTlsGet              10002cd1 f   socket_md.obj
 0001:00001cdc       _dbgsysTlsPut              10002cdc f   socket_md.obj
 0001:00001ceb       ___WSAFDIsSet@8            10002ceb f   ws2_32:WS2_32.dll
 0001:00001cf1       ___raise_securityfailure   10002cf1 f   MSVCRT:gs_report.obj
 0001:00001d19       ___report_gsfailure        10002d19 f   MSVCRT:gs_report.obj
 0001:00001e12       ___report_rangecheckfailure 10002e12 f   MSVCRT:gs_report.obj
 0001:00001e1e       ___report_securityfailure  10002e1e f   MSVCRT:gs_report.obj
 0001:00001eec       @__security_check_cookie@4 10002eec f   MSVCRT:secchk.obj
 0001:00001f00       __alldiv                   10002f00 f   MSVCRT:lldiv.obj
 0001:000022ea       __DllMainCRTStartup@12     100032ea f   MSVCRT:dll_dllmain.obj
 0001:0000235a       ___security_init_cookie    1000335a f   MSVCRT:gs_support.obj
 0001:000023a5       ?__scrt_initialize_type_info@@YAXXZ 100033a5 f   MSVCRT:tncleanup.obj
 0001:000023b1       ?__scrt_uninitialize_type_info@@YAXXZ 100033b1 f   MSVCRT:tncleanup.obj
 0001:000023bd       ___local_stdio_scanf_options 100033bd f i MSVCRT:default_local_stdio_options.obj
 0001:000023c3       ___scrt_initialize_default_local_stdio_options 100033c3 f   MSVCRT:default_local_stdio_options.obj
 0001:00002424       ___scrt_acquire_startup_lock 10003424 f   MSVCRT:utility.obj
 0001:00002456       ___scrt_dllmain_after_initialize_c 10003456 f   MSVCRT:utility.obj
 0001:00002481       ___scrt_dllmain_before_initialize_c 10003481 f   MSVCRT:utility.obj
 0001:0000248f       ___scrt_dllmain_crt_thread_attach 1000348f f   MSVCRT:utility.obj
 0001:000024ae       ___scrt_dllmain_crt_thread_detach 100034ae f   MSVCRT:utility.obj
 0001:000024bb       ___scrt_dllmain_exception_filter 100034bb f   MSVCRT:utility.obj
 0001:000024ef       ___scrt_dllmain_uninitialize_c 100034ef f   MSVCRT:utility.obj
 0001:00002512       ___scrt_dllmain_uninitialize_critical 10003512 f   MSVCRT:utility.obj
 0001:0000251f       ___scrt_initialize_crt     1000351f f   MSVCRT:utility.obj
 0001:00002558       ___scrt_initialize_onexit_tables 10003558 f   MSVCRT:utility.obj
 0001:000025df       ___scrt_is_nonwritable_in_current_image 100035df f   MSVCRT:utility.obj
 0001:00002673       ___scrt_release_startup_lock 10003673 f   MSVCRT:utility.obj
 0001:00002690       ___scrt_uninitialize_crt   10003690 f   MSVCRT:utility.obj
 0001:000026b8       ___scrt_get_dyn_tls_init_callback 100036b8 f   MSVCRT:dyn_tls_init.obj
 0001:000026be       ___scrt_fastfail           100036be f   MSVCRT:utility_desktop.obj
 0001:000027d8       __crt_debugger_hook        100037d8 f   MSVCRT:utility_desktop.obj
 0001:000027e0       __RTC_Initialize           100037e0 f   MSVCRT:initsect.obj
 0001:0000280c       __RTC_Terminate            1000380c f   MSVCRT:initsect.obj
 0001:00002840       __SEH_prolog4              10003840 f   MSVCRT:sehprolg4.obj
 0001:00002884       __SEH_epilog4              10003884 f   MSVCRT:sehprolg4.obj
 0001:00002898       __except_handler4          10003898 f   MSVCRT:chandler4gs.obj
 0001:000028c7       @_guard_check_icall_nop@4  100038c7 f i MSVCRT:guard_support.obj
 0001:000028ca       ___isa_available_init      100038ca f   MSVCRT:cpu_disp.obj
 0001:00002a9a       __get_startup_argv_mode    10003a9a f   MSVCRT:argv_mode.obj
 0001:00002a9e       ___scrt_is_ucrt_dll_in_use 10003a9e f   MSVCRT:ucrt_detection.obj
 0001:00002aaa       _IsProcessorFeaturePresent@4 10003aaa f   kernel32:KERNEL32.dll
 0001:00002ab0       _memcmp                    10003ab0 f   vcruntime:VCRUNTIME140.dll
 0001:00002ab6       _memcpy                    10003ab6 f   vcruntime:VCRUNTIME140.dll
 0001:00002abc       _memset                    10003abc f   vcruntime:VCRUNTIME140.dll
 0001:00002ac2       _strchr                    10003ac2 f   vcruntime:VCRUNTIME140.dll
 0001:00002ac8       _strrchr                   10003ac8 f   vcruntime:VCRUNTIME140.dll
 0001:00002ace       ___std_type_info_destroy_list 10003ace f   vcruntime:VCRUNTIME140.dll
 0001:00002ad4       __except_handler4_common   10003ad4 f   vcruntime:VCRUNTIME140.dll
 0001:00002ada       _strcat                    10003ada f   ucrt:api-ms-win-crt-string-l1-1-0.dll
 0001:00002ae0       _strcmp                    10003ae0 f   ucrt:api-ms-win-crt-string-l1-1-0.dll
 0001:00002ae6       _strcpy                    10003ae6 f   ucrt:api-ms-win-crt-string-l1-1-0.dll
 0001:00002aec       _strlen                    10003aec f   ucrt:api-ms-win-crt-string-l1-1-0.dll
 0001:00002af2       __initterm                 10003af2 f   ucrt:api-ms-win-crt-runtime-l1-1-0.dll
 0001:00002af8       __initterm_e               10003af8 f   ucrt:api-ms-win-crt-runtime-l1-1-0.dll
 0001:00002afe       __seh_filter_dll           10003afe f   ucrt:api-ms-win-crt-runtime-l1-1-0.dll
 0001:00002b04       __configure_narrow_argv    10003b04 f   ucrt:api-ms-win-crt-runtime-l1-1-0.dll
 0001:00002b0a       __initialize_narrow_environment 10003b0a f   ucrt:api-ms-win-crt-runtime-l1-1-0.dll
 0001:00002b10       __initialize_onexit_table  10003b10 f   ucrt:api-ms-win-crt-runtime-l1-1-0.dll
 0001:00002b16       __execute_onexit_table     10003b16 f   ucrt:api-ms-win-crt-runtime-l1-1-0.dll
 0001:00002b1c       __cexit                    10003b1c f   ucrt:api-ms-win-crt-runtime-l1-1-0.dll
 0001:00002b22       ___scrt_stub_for_acrt_initialize 10003b22 f   MSVCRT:ucrt_stubs.obj
 0001:00002b22       ___acrt_thread_detach      10003b22 f   MSVCRT:ucrt_stubs.obj
 0001:00002b22       ___vcrt_thread_detach      10003b22 f   MSVCRT:ucrt_stubs.obj
 0001:00002b22       ___acrt_uninitialize       10003b22 f   MSVCRT:ucrt_stubs.obj
 0001:00002b22       ___vcrt_uninitialize_critical 10003b22 f   MSVCRT:ucrt_stubs.obj
 0001:00002b22       ___acrt_thread_attach      10003b22 f   MSVCRT:ucrt_stubs.obj
 0001:00002b22       ___scrt_stub_for_acrt_uninitialize 10003b22 f   MSVCRT:ucrt_stubs.obj
 0001:00002b22       ___vcrt_thread_attach      10003b22 f   MSVCRT:ucrt_stubs.obj
 0001:00002b22       ___acrt_initialize         10003b22 f   MSVCRT:ucrt_stubs.obj
 0001:00002b22       ___scrt_stub_for_acrt_thread_detach 10003b22 f   MSVCRT:ucrt_stubs.obj
 0001:00002b22       ___scrt_stub_for_acrt_uninitialize_critical 10003b22 f   MSVCRT:ucrt_stubs.obj
 0001:00002b22       ___vcrt_initialize         10003b22 f   MSVCRT:ucrt_stubs.obj
 0001:00002b22       ___scrt_stub_for_acrt_thread_attach 10003b22 f   MSVCRT:ucrt_stubs.obj
 0001:00002b22       ___vcrt_uninitialize       10003b22 f   MSVCRT:ucrt_stubs.obj
 0001:00002b22       ___acrt_uninitialize_critical 10003b22 f   MSVCRT:ucrt_stubs.obj
 0001:00002b25       ___scrt_stub_for_is_c_termination_complete 10003b25 f   MSVCRT:ucrt_stubs.obj
 0001:00002b25       __is_c_termination_complete 10003b25 f   MSVCRT:ucrt_stubs.obj
 0001:00002b28       __filter_x86_sse2_floating_point_exception_default 10003b28 f   MSVCRT:x86_exception_filter.obj
 0001:00002b28       __filter_x86_sse2_floating_point_exception 10003b28 f   MSVCRT:x86_exception_filter.obj
 0002:00000000       __imp__if_nametoindex@4    10004000     iphlpapi:IPHLPAPI.DLL
 0002:00000004       \177IPHLPAPI_NULL_THUNK_DATA 10004004     iphlpapi:IPHLPAPI.DLL
 0002:00000008       __imp__IsDebuggerPresent@0 10004008     kernel32:KERNEL32.dll
 0002:0000000c       __imp__InitializeSListHead@4 1000400c     kernel32:KERNEL32.dll
 0002:00000010       __imp__GetSystemTimeAsFileTime@4 10004010     kernel32:KERNEL32.dll
 0002:00000014       __imp__GetCurrentThreadId@0 10004014     kernel32:KERNEL32.dll
 0002:00000018       __imp__GetCurrentProcessId@0 10004018     kernel32:KERNEL32.dll
 0002:0000001c       __imp__IsProcessorFeaturePresent@4 1000401c     kernel32:KERNEL32.dll
 0002:00000020       __imp__TerminateProcess@8  10004020     kernel32:KERNEL32.dll
 0002:00000024       __imp__GetCurrentProcess@0 10004024     kernel32:KERNEL32.dll
 0002:00000028       __imp__UnhandledExceptionFilter@4 10004028     kernel32:KERNEL32.dll
 0002:0000002c       __imp__SystemTimeToFileTime@8 1000402c     kernel32:KERNEL32.dll
 0002:00000030       __imp__GetSystemTime@4     10004030     kernel32:KERNEL32.dll
 0002:00000034       __imp__TlsSetValue@8       10004034     kernel32:KERNEL32.dll
 0002:00000038       __imp__TlsGetValue@4       10004038     kernel32:KERNEL32.dll
 0002:0000003c       __imp__TlsAlloc@0          1000403c     kernel32:KERNEL32.dll
 0002:00000040       __imp__SetHandleInformation@12 10004040     kernel32:KERNEL32.dll
 0002:00000044       __imp__QueryPerformanceCounter@4 10004044     kernel32:KERNEL32.dll
 0002:00000048       __imp__SetUnhandledExceptionFilter@4 10004048     kernel32:KERNEL32.dll
 0002:0000004c       \177KERNEL32_NULL_THUNK_DATA 1000404c     kernel32:KERNEL32.dll
 0002:00000050       __imp____std_type_info_destroy_list 10004050     vcruntime:VCRUNTIME140.dll
 0002:00000054       __imp__strrchr             10004054     vcruntime:VCRUNTIME140.dll
 0002:00000058       __imp__strchr              10004058     vcruntime:VCRUNTIME140.dll
 0002:0000005c       __imp__memset              1000405c     vcruntime:VCRUNTIME140.dll
 0002:00000060       __imp__memcpy              10004060     vcruntime:VCRUNTIME140.dll
 0002:00000064       __imp__memcmp              10004064     vcruntime:VCRUNTIME140.dll
 0002:00000068       __imp___except_handler4_common 10004068     vcruntime:VCRUNTIME140.dll
 0002:0000006c       \177VCRUNTIME140_NULL_THUNK_DATA 1000406c     vcruntime:VCRUNTIME140.dll
 0002:00000070       __imp__recv@16             10004070     ws2_32:WS2_32.dll
 0002:00000074       __imp__ntohs@4             10004074     ws2_32:WS2_32.dll
 0002:00000078       __imp__ntohl@4             10004078     ws2_32:WS2_32.dll
 0002:0000007c       __imp__listen@8            1000407c     ws2_32:WS2_32.dll
 0002:00000080       __imp__htons@4             10004080     ws2_32:WS2_32.dll
 0002:00000084       __imp__htonl@4             10004084     ws2_32:WS2_32.dll
 0002:00000088       __imp__getsockopt@20       10004088     ws2_32:WS2_32.dll
 0002:0000008c       __imp__send@16             1000408c     ws2_32:WS2_32.dll
 0002:00000090       __imp__ioctlsocket@12      10004090     ws2_32:WS2_32.dll
 0002:00000094       __imp__connect@12          10004094     ws2_32:WS2_32.dll
 0002:00000098       __imp__setsockopt@20       10004098     ws2_32:WS2_32.dll
 0002:0000009c       __imp__closesocket@4       1000409c     ws2_32:WS2_32.dll
 0002:000000a0       __imp__bind@12             100040a0     ws2_32:WS2_32.dll
 0002:000000a4       __imp__accept@12           100040a4     ws2_32:WS2_32.dll
 0002:000000a8       __imp____WSAFDIsSet@8      100040a8     ws2_32:WS2_32.dll
 0002:000000ac       __imp__inet_pton@12        100040ac     ws2_32:WS2_32.dll
 0002:000000b0       __imp__getnameinfo@28      100040b0     ws2_32:WS2_32.dll
 0002:000000b4       __imp__freeaddrinfo@4      100040b4     ws2_32:WS2_32.dll
 0002:000000b8       __imp__select@20           100040b8     ws2_32:WS2_32.dll
 0002:000000bc       __imp__getaddrinfo@16      100040bc     ws2_32:WS2_32.dll
 0002:000000c0       __imp__WSAGetLastError@0   100040c0     ws2_32:WS2_32.dll
 0002:000000c4       __imp__WSACleanup@0        100040c4     ws2_32:WS2_32.dll
 0002:000000c8       __imp__WSAStartup@8        100040c8     ws2_32:WS2_32.dll
 0002:000000cc       __imp__getprotobyname@4    100040cc     ws2_32:WS2_32.dll
 0002:000000d0       __imp__socket@12           100040d0     ws2_32:WS2_32.dll
 0002:000000d4       __imp__getsockname@12      100040d4     ws2_32:WS2_32.dll
 0002:000000d8       __imp__shutdown@8          100040d8     ws2_32:WS2_32.dll
 0002:000000dc       \177WS2_32_NULL_THUNK_DATA 100040dc     ws2_32:WS2_32.dll
 0002:000000e0       __imp__strtoul             100040e0     ucrt:api-ms-win-crt-convert-l1-1-0.dll
 0002:000000e4       \177api-ms-win-crt-convert-l1-1-0_NULL_THUNK_DATA 100040e4     ucrt:api-ms-win-crt-convert-l1-1-0.dll
 0002:000000e8       __imp___cexit              100040e8     ucrt:api-ms-win-crt-runtime-l1-1-0.dll
 0002:000000ec       __imp___execute_onexit_table 100040ec     ucrt:api-ms-win-crt-runtime-l1-1-0.dll
 0002:000000f0       __imp___initialize_onexit_table 100040f0     ucrt:api-ms-win-crt-runtime-l1-1-0.dll
 0002:000000f4       __imp___initialize_narrow_environment 100040f4     ucrt:api-ms-win-crt-runtime-l1-1-0.dll
 0002:000000f8       __imp___initterm           100040f8     ucrt:api-ms-win-crt-runtime-l1-1-0.dll
 0002:000000fc       __imp___initterm_e         100040fc     ucrt:api-ms-win-crt-runtime-l1-1-0.dll
 0002:00000100       __imp___seh_filter_dll     10004100     ucrt:api-ms-win-crt-runtime-l1-1-0.dll
 0002:00000104       __imp___configure_narrow_argv 10004104     ucrt:api-ms-win-crt-runtime-l1-1-0.dll
 0002:00000108       \177api-ms-win-crt-runtime-l1-1-0_NULL_THUNK_DATA 10004108     ucrt:api-ms-win-crt-runtime-l1-1-0.dll
 0002:0000010c       __imp____acrt_iob_func     1000410c     ucrt:api-ms-win-crt-stdio-l1-1-0.dll
 0002:00000110       __imp____stdio_common_vfprintf 10004110     ucrt:api-ms-win-crt-stdio-l1-1-0.dll
 0002:00000114       __imp____stdio_common_vsprintf 10004114     ucrt:api-ms-win-crt-stdio-l1-1-0.dll
 0002:00000118       \177api-ms-win-crt-stdio-l1-1-0_NULL_THUNK_DATA 10004118     ucrt:api-ms-win-crt-stdio-l1-1-0.dll
 0002:0000011c       __imp__strcpy              1000411c     ucrt:api-ms-win-crt-string-l1-1-0.dll
 0002:00000120       __imp__strlen              10004120     ucrt:api-ms-win-crt-string-l1-1-0.dll
 0002:00000124       __imp__strcat              10004124     ucrt:api-ms-win-crt-string-l1-1-0.dll
 0002:00000128       __imp__strpbrk             10004128     ucrt:api-ms-win-crt-string-l1-1-0.dll
 0002:0000012c       __imp__strncmp             1000412c     ucrt:api-ms-win-crt-string-l1-1-0.dll
 0002:00000130       __imp__strcmp              10004130     ucrt:api-ms-win-crt-string-l1-1-0.dll
 0002:00000134       \177api-ms-win-crt-string-l1-1-0_NULL_THUNK_DATA 10004134     ucrt:api-ms-win-crt-string-l1-1-0.dll
 0002:00000138       ___guard_check_icall_fptr  10004138     MSVCRT:guard_support.obj
 0002:0000013c       ___xc_a                    1000413c     MSVCRT:initializers.obj
 0002:00000140       ___xc_z                    10004140     MSVCRT:initializers.obj
 0002:00000144       ___xi_a                    10004144     MSVCRT:initializers.obj
 0002:00000148       ___xi_z                    10004148     MSVCRT:initializers.obj
 0002:0000014c       ___xp_a                    1000414c     MSVCRT:initializers.obj
 0002:00000150       ___xp_z                    10004150     MSVCRT:initializers.obj
 0002:00000154       ___xt_a                    10004154     MSVCRT:initializers.obj
 0002:00000158       ___xt_z                    10004158     MSVCRT:initializers.obj
 0002:00000160       ??_C@_02LMMGGCAJ@?3?5@     10004160     socketTransport.obj
 0002:00000164       ??_C@_0BN@KHJBBJDI@setsockopt?5TCPNODELAY?5failed@ 10004164     socketTransport.obj
 0002:00000184       ??_C@_0BP@DIBLKMHJ@setsockopt?5SO_REUSEADDR?5failed@ 10004184     socketTransport.obj
 0002:000001a4       ??_C@_0P@FPMMELAG@JDWP?9Handshake@ 100041a4     socketTransport.obj
 0002:000001b4       ??_C@_0BJ@GINIINMB@timeout?5during?5handshake@ 100041b4     socketTransport.obj
 0002:000001d0       ??_C@_0DC@PHHFHFJN@handshake?5failed?5?9?5connection?5p@ 100041d0     socketTransport.obj
 0002:00000204       ??_C@_0BN@NDCFIPML@recv?5failed?5during?5handshake@ 10004204     socketTransport.obj
 0002:00000224       ??_C@_0DB@KBPJCIBD@handshake?5failed?5?9?5received?5?$DO?$CFs@ 10004224     socketTransport.obj
 0002:00000258       ??_C@_0BN@MCHFOAHG@send?5failed?5during?5handshake@ 10004258     socketTransport.obj
 0002:00000278       ??_C@_0BG@JDCCCDJP@failed?5to?5parse?5scope@ 10004278     socketTransport.obj
 0002:00000290       ??_C@_0O@BNNCBLEN@out?5of?5memory@ 10004290     socketTransport.obj
 0002:000002a0       ??_C@_0CF@ELCCDBKH@getaddrinfo?3?5failed?5to?5parse?5ad@ 100042a0     socketTransport.obj
 0002:000002c8       ??_C@_0CC@BPMEHIMC@IPv4?5address?5cannot?5contain?5sco@ 100042c8     socketTransport.obj
 0002:000002ec       ??_C@_0BO@EGDNNDCF@invalid?5port?5number?5specified@ 100042ec     socketTransport.obj
 0002:0000030c       ??_C@_02EFNPNKFJ@?1?$CL@   1000430c     socketTransport.obj
 0002:00000310       ??_C@_0BN@JKPNAKGA@Error?5in?5allow?5option?3?5?8?$CFs?8?6@ 10004310     socketTransport.obj
 0002:00000330       ??_C@_0CD@EIJBPJF@invalid?5IP?5address?5in?5allow?5opt@ 10004330     socketTransport.obj
 0002:00000354       ??_C@_0CA@GFDOAML@invalid?5netmask?5in?5allow?5option@ 10004354     socketTransport.obj
 0002:00000374       ??_C@_0BH@HKLPKFAI@socket?5creation?5failed@ 10004374     socketTransport.obj
 0002:0000038c       ??_C@_0M@NNJMLKEI@bind?5failed@ 1000438c     socketTransport.obj
 0002:00000398       ??_C@_0O@MHKNJCGE@listen?5failed@ 10004398     socketTransport.obj
 0002:000003a8       ??_C@_0BD@PDGFKJCK@getsockname?5failed@ 100043a8     socketTransport.obj
 0002:000003bc       ??_C@_02DPKJAMEF@?$CFd@    100043bc     socketTransport.obj
 0002:000003c0       ??_C@_01GBGANLPD@0@        100043c0     socketTransport.obj
 0002:000003c4       ??_C@_0BN@KALBAHGL@listen?5failed?3?5wrong?5address@ 100043c4     socketTransport.obj
 0002:000003e4       ??_C@_0P@DBOBDCFH@?3?3ffff?30?40?40?40@ 100043e4     socketTransport.obj
 0002:000003f4       ??_C@_0M@GKCHHBEN@poll?5failed@ 100043f4     socketTransport.obj
 0002:00000400       ??_C@_0CB@LPJGLJKP@timed?5out?5waiting?5for?5connectio@ 10004400     socketTransport.obj
 0002:00000424       ??_C@_0O@NBABPAKN@accept?5failed@ 10004424     socketTransport.obj
 0002:00000434       ??_C@_0O@MEOPDPBI@?$DMbad?5address?$DO@ 10004434     socketTransport.obj
 0002:00000444       ??_C@_0CI@EAPIJEBA@ERROR?3?5Peer?5not?5allowed?5to?5conn@ 10004444     socketTransport.obj
 0002:0000046c       ??_C@_0BP@FADEKCPP@Debugger?5failed?5to?5attach?3?5?$CFs?6@ 1000446c     socketTransport.obj
 0002:0000048c       ??_C@_0CI@IHMKOBEI@timeout?5waiting?5for?5debugger?5to@ 1000448c     socketTransport.obj
 0002:000004b4       ??_C@_0BE@KOKKGIKP@connection?5not?5open@ 100044b4     socketTransport.obj
 0002:000004c8       ??_C@_0N@NOKLILHD@close?5failed@ 100044c8     socketTransport.obj
 0002:000004d8       ??_C@_0BI@PPNDHPPD@unable?5to?5create?5socket@ 100044d8     socketTransport.obj
 0002:000004f0       ??_C@_0BC@DJFNFCAI@connect?5timed?5out@ 100044f0     socketTransport.obj
 0002:00000504       ??_C@_0P@FKKLKLOM@connect?5failed@ 10004504     socketTransport.obj
 0002:00000514       ??_C@_0BD@CJKAJNDH@address?5is?5missing@ 10004514     socketTransport.obj
 0002:00000528       ??_C@_0P@KCFPLCED@packet?5is?5NULL@ 10004528     socketTransport.obj
 0002:00000538       ??_C@_0P@BHAFPBHF@invalid?5length@ 10004538     socketTransport.obj
 0002:00000548       ??_C@_0M@EADLIJBM@send?5failed@ 10004548     socketTransport.obj
 0002:00000554       ??_C@_0P@GOGFFADL@packet?5is?5null@ 10004554     socketTransport.obj
 0002:00000564       ??_C@_0O@NBMIKEGI@premature?5EOF@ 10004564     socketTransport.obj
 0002:00000574       ??_C@_0L@IBALKEMH@recv?5error@ 10004574     socketTransport.obj
 0002:00000580       ??_C@_0CO@MNFHICJC@Badly?5formed?5packet?5received?5?9?5@ 10004580     socketTransport.obj
 0002:000005b0       ??_C@_0DD@BGKOFAPC@NULL?5pointer?5to?5transport?5confi@ 100045b0     socketTransport.obj
 0002:000005e4       ??_C@_0CB@MLDNKOMM@allow?5option?5should?5not?5be?5empt@ 100045e4     socketTransport.obj
 0002:00000608       ??_C@_0CE@MKEKLDBI@allow?5option?5?8?$CK?8?5cannot?5be?5expa@ 10004608     socketTransport.obj
 0002:0000062c       ??_C@_04LOAJBDKD@true@     1000462c     socketTransport.obj
 0002:00000634       ??_C@_05LAPONLG@false@     10004634     socketTransport.obj
 0002:0000063c       ??_C@_0BB@NAICLKDB@java?1lang?1System@ 1000463c     socketTransport.obj
 0002:00000650       ??_C@_0CH@NCPCFFHJ@?$CILjava?1lang?1String?$DL?$CJLjava?1lang?1@ 10004650     socketTransport.obj
 0002:00000678       ??_C@_0M@NBNLNHMA@getProperty@ 10004678     socketTransport.obj
 0002:00000684       ??_C@_0BJ@OCGKBLBN@java?4net?4preferIPv4Stack@ 10004684     socketTransport.obj
 0002:000006a0       ??_C@_0BN@IKFECHDC@java?4net?4preferIPv6Addresses@ 100046a0     socketTransport.obj
 0002:00000830       ??_C@_0DE@NDGANADE@Provider?5initialization?5failed?5@ 10004830     socket_md.obj
 0002:00000864       ??_C@_0BC@HFNFNKAI@Permission?5denied@ 10004864     socket_md.obj
 0002:00000878       ??_C@_0BH@LOKACPE@Address?5already?5in?5use@ 10004878     socket_md.obj
 0002:00000890       ??_C@_0CA@NBHADPNL@Cannot?5assign?5requested?5address@ 10004890     socket_md.obj
 0002:000008b0       ??_C@_0DA@KDGLCJJO@Address?5family?5not?5supported?5by@ 100048b0     socket_md.obj
 0002:000008e0       ??_C@_0BO@BMABNIPB@Operation?5already?5in?5progress@ 100048e0     socket_md.obj
 0002:00000900       ??_C@_0CB@DJAOADN@Software?5caused?5connection?5abor@ 10004900     socket_md.obj
 0002:00000924       ??_C@_0BD@NPDMPPFP@Connection?5refused@ 10004924     socket_md.obj
 0002:00000938       ??_C@_0BJ@FJAMCHKE@Connection?5reset?5by?5peer@ 10004938     socket_md.obj
 0002:00000954       ??_C@_0BN@HFCIEIME@Destination?5address?5required@ 10004954     socket_md.obj
 0002:00000974       ??_C@_0M@LOEHLCJD@Bad?5address@ 10004974     socket_md.obj
 0002:00000980       ??_C@_0N@OHOPOBEF@Host?5is?5down@ 10004980     socket_md.obj
 0002:00000990       ??_C@_0BB@PFBILCPA@No?5route?5to?5host@ 10004990     socket_md.obj
 0002:000009a4       ??_C@_0BK@LBMNDGCG@Operation?5now?5in?5progress@ 100049a4     socket_md.obj
 0002:000009c0       ??_C@_0BK@FJBOAFDK@Interrupted?5function?5call@ 100049c0     socket_md.obj
 0002:000009dc       ??_C@_0BB@HMGGCEBG@Invalid?5argument@ 100049dc     socket_md.obj
 0002:000009f0       ??_C@_0BM@CCONNCKE@Socket?5is?5already?5connected@ 100049f0     socket_md.obj
 0002:00000a0c       ??_C@_0BE@INBJMKGG@Too?5many?5open?5files@ 10004a0c     socket_md.obj
 0002:00000a20       ??_C@_0EN@MMGGBIMI@The?5message?5is?5larger?5than?5the?5@ 10004a20     socket_md.obj
 0002:00000a70       ??_C@_0BA@LPIEBGEK@Network?5is?5down@ 10004a70     socket_md.obj
 0002:00000a80       ??_C@_0CE@JHDCOCF@Network?5dropped?5connection?5on?5r@ 10004a80     socket_md.obj
 0002:00000aa4       ??_C@_0BH@CIEOBPFM@Network?5is?5unreachable@ 10004aa4     socket_md.obj
 0002:00000abc       ??_C@_0DJ@FJOKEEBP@No?5buffer?5space?5available?5?$CImaxi@ 10004abc     socket_md.obj
 0002:00000af8       ??_C@_0BE@NEGCDJON@Bad?5protocol?5option@ 10004af8     socket_md.obj
 0002:00000b0c       ??_C@_0BI@ILAOGBJJ@Socket?5is?5not?5connected@ 10004b0c     socket_md.obj
 0002:00000b24       ??_C@_0BO@PFGGHOGH@Socket?5operation?5on?5nonsocket@ 10004b24     socket_md.obj
 0002:00000b44       ??_C@_0BI@EDJAHLMH@Operation?5not?5supported@ 10004b44     socket_md.obj
 0002:00000b5c       ??_C@_0BO@EBCCBLCJ@Protocol?5family?5not?5supported@ 10004b5c     socket_md.obj
 0002:00000b7c       ??_C@_0BD@LPHIGPM@Too?5many?5processes@ 10004b7c     socket_md.obj
 0002:00000b90       ??_C@_0BH@JNBKLLAJ@Protocol?5not?5supported@ 10004b90     socket_md.obj
 0002:00000ba8       ??_C@_0BP@PDKJLOAE@Protocol?5wrong?5type?5for?5socket@ 10004ba8     socket_md.obj
 0002:00000bc8       ??_C@_0CC@DAIJOIKC@Cannot?5send?5after?5socket?5shutdo@ 10004bc8     socket_md.obj
 0002:00000bec       ??_C@_0BK@LMAIHBL@Socket?5type?5not?5supported@ 10004bec     socket_md.obj
 0002:00000c08       ??_C@_0BF@IBBHAGLD@Connection?5timed?5out@ 10004c08     socket_md.obj
 0002:00000c20       ??_C@_0BF@EHICFGGJ@Class?5type?5not?5found@ 10004c20     socket_md.obj
 0002:00000c38       ??_C@_0CB@EPFKGNAK@Resource?5temporarily?5unavailabl@ 10004c38     socket_md.obj
 0002:00000c5c       ??_C@_0P@CAFMJNJH@Host?5not?5found@ 10004c5c     socket_md.obj
 0002:00000c6c       ??_C@_0BO@GICNLCFB@Insufficient?5memory?5available@ 10004c6c     socket_md.obj
 0002:00000c8c       ??_C@_0CI@CFJNLLNI@Successful?5WSAStartup?5not?5yet?5p@ 10004c8c     socket_md.obj
 0002:00000cb4       ??_C@_0CN@KFPNHBIN@Valid?5name?0?5no?5data?5record?5of?5r@ 10004cb4     socket_md.obj
 0002:00000ce4       ??_C@_0BP@BOOHLDLA@This?5is?5a?5nonrecoverable?5error@ 10004ce4     socket_md.obj
 0002:00000d04       ??_C@_0CB@PLJNFILF@Network?5subsystem?5is?5unavailabl@ 10004d04     socket_md.obj
 0002:00000d28       ??_C@_0CA@DOKOCCFB@Nonauthoritative?5host?5not?5found@ 10004d28     socket_md.obj
 0002:00000d48       ??_C@_0CB@GHMLGJBG@Winsock?4dll?5version?5out?5of?5rang@ 10004d48     socket_md.obj
 0002:00000d6c       ??_C@_0BO@ILFFGILJ@Graceful?5shutdown?5in?5progress@ 10004d6c     socket_md.obj
 0002:00000d8c       ??_C@_0BN@KGMIDOOK@Overlapped?5operation?5aborted@ 10004d8c     socket_md.obj
 0002:00000dac       ??_C@_03FCLDNGNL@TCP@      10004dac     socket_md.obj
 0002:00000db0       ??_C@_0BB@IDELEPKG@winsock?5error?5?$CFd@ 10004db0     socket_md.obj
 0002:00000dc4       _in6addr_any               10004dc4     ws2_32:indef.obj
 0002:00000ddc       __pDefaultRawDllMain       10004ddc     MSVCRT:dll_dllmain.obj
 0002:00000ddc       __pRawDllMain              10004ddc     MSVCRT:dll_dllmain.obj
 0002:00000e50       __load_config_used         10004e50     MSVCRT:loadcfg.obj
 0002:00000f08       ___safe_se_handler_table   10004f08     <linker-defined>
 0002:00001194       ___rtc_iaa                 10005194     MSVCRT:initsect.obj
 0002:00001198       ___rtc_izz                 10005198     MSVCRT:initsect.obj
 0002:0000119c       ___rtc_taa                 1000519c     MSVCRT:initsect.obj
 0002:000011a0       ___rtc_tzz                 100051a0     MSVCRT:initsect.obj
 0002:0000128c       __IMPORT_DESCRIPTOR_WS2_32 1000528c     ws2_32:WS2_32.dll
 0002:000012a0       __IMPORT_DESCRIPTOR_IPHLPAPI 100052a0     iphlpapi:IPHLPAPI.DLL
 0002:000012b4       __IMPORT_DESCRIPTOR_KERNEL32 100052b4     kernel32:KERNEL32.dll
 0002:000012c8       __IMPORT_DESCRIPTOR_VCRUNTIME140 100052c8     vcruntime:VCRUNTIME140.dll
 0002:000012dc       __IMPORT_DESCRIPTOR_api-ms-win-crt-stdio-l1-1-0 100052dc     ucrt:api-ms-win-crt-stdio-l1-1-0.dll
 0002:000012f0       __IMPORT_DESCRIPTOR_api-ms-win-crt-string-l1-1-0 100052f0     ucrt:api-ms-win-crt-string-l1-1-0.dll
 0002:00001304       __IMPORT_DESCRIPTOR_api-ms-win-crt-convert-l1-1-0 10005304     ucrt:api-ms-win-crt-convert-l1-1-0.dll
 0002:00001318       __IMPORT_DESCRIPTOR_api-ms-win-crt-runtime-l1-1-0 10005318     ucrt:api-ms-win-crt-runtime-l1-1-0.dll
 0002:0000132c       __NULL_IMPORT_DESCRIPTOR   1000532c     ws2_32:WS2_32.dll
 0003:00000010       ___security_cookie_complement 10006010     MSVCRT:gs_cookie.obj
 0003:00000014       ___security_cookie         10006014     MSVCRT:gs_cookie.obj
 0003:00000020       ___scrt_native_dllmain_reason 10006020     MSVCRT:utility.obj
 0003:00000030       ___isa_enabled             10006030     MSVCRT:cpu_disp.obj
 0003:00000034       ___scrt_ucrt_dll_is_in_use 10006034     MSVCRT:ucrt_stubs.obj
 0003:000007a8       ?__type_info_root_node@@3U__type_info_node@@A 100067a8     MSVCRT:tncleanup.obj
 0003:000007b0       ?_OptionsStorage@?1??__local_stdio_scanf_options@@9@4_KA 100067b0     MSVCRT:default_local_stdio_options.obj
 0003:000007b8       ___scrt_current_native_startup_state 100067b8     MSVCRT:utility.obj
 0003:000007bc       ___scrt_native_startup_lock 100067bc     MSVCRT:utility.obj
 0003:000007dc       ___scrt_debugger_hook_flag 100067dc     MSVCRT:utility_desktop.obj
 0003:000007e0       ___isa_available           100067e0     MSVCRT:cpu_disp.obj
 0003:000007e4       ___favor                   100067e4     MSVCRT:cpu_disp.obj
 0003:000007e8       ?_OptionsStorage@?1??__local_stdio_printf_options@@9@9 100067e8     <common>
 0003:000007f0       ___dyn_tls_init_callback   100067f0     <common>

 entry point at        0001:000022ea

 Static symbols

 0000:ffff7000       .debug$S                   10000000     dt_socket.exp
 0000:ffff7000       .debug$S                   10000000     vcruntime:VCRUNTIME140.dll
 0000:ffff7000       .debug$S                   10000000     vcruntime:VCRUNTIME140.dll
 0000:ffff7000       .debug$S                   10000000     vcruntime:VCRUNTIME140.dll
 0000:ffff7000       .debug$S                   10000000     vcruntime:VCRUNTIME140.dll
 0000:ffff7000       .debug$S                   10000000     vcruntime:VCRUNTIME140.dll
 0000:ffff7000       .debug$S                   10000000     vcruntime:VCRUNTIME140.dll
 0000:ffff7000       .debug$S                   10000000     vcruntime:VCRUNTIME140.dll
 0000:ffff7000       .debug$S                   10000000     vcruntime:VCRUNTIME140.dll
 0000:ffff7000       .debug$S                   10000000     vcruntime:VCRUNTIME140.dll
 0000:ffff7000       .debug$S                   10000000     ucrt:api-ms-win-crt-convert-l1-1-0.dll
 0000:ffff7000       .debug$S                   10000000     ucrt:api-ms-win-crt-runtime-l1-1-0.dll
 0000:ffff7000       .debug$S                   10000000     ucrt:api-ms-win-crt-runtime-l1-1-0.dll
 0000:ffff7000       .debug$S                   10000000     ucrt:api-ms-win-crt-runtime-l1-1-0.dll
 0000:ffff7000       .debug$S                   10000000     ucrt:api-ms-win-crt-runtime-l1-1-0.dll
 0000:ffff7000       .debug$S                   10000000     ucrt:api-ms-win-crt-runtime-l1-1-0.dll
 0000:ffff7000       .debug$S                   10000000     ucrt:api-ms-win-crt-runtime-l1-1-0.dll
 0000:ffff7000       .debug$S                   10000000     ucrt:api-ms-win-crt-runtime-l1-1-0.dll
 0000:ffff7000       .debug$S                   10000000     ucrt:api-ms-win-crt-runtime-l1-1-0.dll
 0000:ffff7000       .debug$S                   10000000     ucrt:api-ms-win-crt-runtime-l1-1-0.dll
 0000:ffff7000       .debug$S                   10000000     ucrt:api-ms-win-crt-runtime-l1-1-0.dll
 0000:ffff7000       .debug$S                   10000000     ucrt:api-ms-win-crt-runtime-l1-1-0.dll
 0000:ffff7000       .debug$S                   10000000     ucrt:api-ms-win-crt-runtime-l1-1-0.dll
 0000:ffff7000       .debug$S                   10000000     ucrt:api-ms-win-crt-stdio-l1-1-0.dll
 0000:ffff7000       .debug$S                   10000000     ucrt:api-ms-win-crt-stdio-l1-1-0.dll
 0000:ffff7000       .debug$S                   10000000     ucrt:api-ms-win-crt-stdio-l1-1-0.dll
 0000:ffff7000       .debug$S                   10000000     ucrt:api-ms-win-crt-string-l1-1-0.dll
 0000:ffff7000       .debug$S                   10000000     ucrt:api-ms-win-crt-string-l1-1-0.dll
 0000:ffff7000       .debug$S                   10000000     ucrt:api-ms-win-crt-string-l1-1-0.dll
 0000:ffff7000       .debug$S                   10000000     ucrt:api-ms-win-crt-string-l1-1-0.dll
 0000:ffff7000       .debug$S                   10000000     ucrt:api-ms-win-crt-string-l1-1-0.dll
 0000:ffff7000       .debug$S                   10000000     ucrt:api-ms-win-crt-string-l1-1-0.dll
 0000:ffff7000       .debug$S                   10000000     iphlpapi:IPHLPAPI.DLL
 0000:ffff7000       .debug$S                   10000000     kernel32:KERNEL32.dll
 0000:ffff7000       .debug$S                   10000000     kernel32:KERNEL32.dll
 0000:ffff7000       .debug$S                   10000000     kernel32:KERNEL32.dll
 0000:ffff7000       .debug$S                   10000000     kernel32:KERNEL32.dll
 0000:ffff7000       .debug$S                   10000000     kernel32:KERNEL32.dll
 0000:ffff7000       .debug$S                   10000000     kernel32:KERNEL32.dll
 0000:ffff7000       .debug$S                   10000000     kernel32:KERNEL32.dll
 0000:ffff7000       .debug$S                   10000000     kernel32:KERNEL32.dll
 0000:ffff7000       .debug$S                   10000000     kernel32:KERNEL32.dll
 0000:ffff7000       .debug$S                   10000000     kernel32:KERNEL32.dll
 0000:ffff7000       .debug$S                   10000000     kernel32:KERNEL32.dll
 0000:ffff7000       .debug$S                   10000000     kernel32:KERNEL32.dll
 0000:ffff7000       .debug$S                   10000000     kernel32:KERNEL32.dll
 0000:ffff7000       .debug$S                   10000000     kernel32:KERNEL32.dll
 0000:ffff7000       .debug$S                   10000000     kernel32:KERNEL32.dll
 0000:ffff7000       .debug$S                   10000000     kernel32:KERNEL32.dll
 0000:ffff7000       .debug$S                   10000000     kernel32:KERNEL32.dll
 0000:ffff7000       .debug$S                   10000000     kernel32:KERNEL32.dll
 0000:ffff7000       .debug$S                   10000000     kernel32:KERNEL32.dll
 0000:ffff7000       .debug$S                   10000000     kernel32:KERNEL32.dll
 0000:ffff7000       .debug$S                   10000000     ws2_32:WS2_32.dll
 0000:ffff7000       .debug$S                   10000000     ws2_32:WS2_32.dll
 0000:ffff7000       .debug$S                   10000000     ws2_32:WS2_32.dll
 0000:ffff7000       .debug$S                   10000000     ws2_32:WS2_32.dll
 0000:ffff7000       .debug$S                   10000000     ws2_32:WS2_32.dll
 0000:ffff7000       .debug$S                   10000000     ws2_32:WS2_32.dll
 0000:ffff7000       .debug$S                   10000000     ws2_32:WS2_32.dll
 0000:ffff7000       .debug$S                   10000000     ws2_32:WS2_32.dll
 0000:ffff7000       .debug$S                   10000000     ws2_32:WS2_32.dll
 0000:ffff7000       .debug$S                   10000000     ws2_32:WS2_32.dll
 0000:ffff7000       .debug$S                   10000000     ws2_32:WS2_32.dll
 0000:ffff7000       .debug$S                   10000000     ws2_32:WS2_32.dll
 0000:ffff7000       .debug$S                   10000000     ws2_32:WS2_32.dll
 0000:ffff7000       .debug$S                   10000000     ws2_32:WS2_32.dll
 0000:ffff7000       .debug$S                   10000000     ws2_32:WS2_32.dll
 0000:ffff7000       .debug$S                   10000000     ws2_32:WS2_32.dll
 0000:ffff7000       .debug$S                   10000000     ws2_32:WS2_32.dll
 0000:ffff7000       .debug$S                   10000000     ws2_32:WS2_32.dll
 0000:ffff7000       .debug$S                   10000000     ws2_32:WS2_32.dll
 0000:ffff7000       .debug$S                   10000000     ws2_32:WS2_32.dll
 0000:ffff7000       .debug$S                   10000000     ws2_32:WS2_32.dll
 0000:ffff7000       .debug$S                   10000000     ws2_32:WS2_32.dll
 0000:ffff7000       .debug$S                   10000000     ws2_32:WS2_32.dll
 0000:ffff7000       .debug$S                   10000000     ws2_32:WS2_32.dll
 0000:ffff7000       .debug$S                   10000000     ws2_32:WS2_32.dll
 0000:ffff7000       .debug$S                   10000000     ws2_32:WS2_32.dll
 0000:ffff7000       .debug$S                   10000000     ws2_32:WS2_32.dll
 0000:ffff7000       .debug$S                   10000000     ws2_32:WS2_32.dll
 0000:ffff7000       .debug$S                   10000000     ws2_32:WS2_32.dll
 0001:0000005d       _connectToAddr             1000105d f   socketTransport.obj
 0001:0000014b       _convertIPv4ToIPv6         1000114b f   socketTransport.obj
 0001:00000190       _getAddrInfo               10001190 f   socketTransport.obj
 0001:00000282       _handshake                 10001282 f   socketTransport.obj
 0001:000003f4       _isEqualIPv6Addr           100013f4 f   socketTransport.obj
 0001:000005c1       _parseAddress              100015c1 f   socketTransport.obj
 0001:000006c7       _parseAllowedAddr          100016c7 f   socketTransport.obj
 0001:00000797       _parseAllowedMask          10001797 f   socketTransport.obj
 0001:00000827       _parseAllowedPeers         10001827 f   socketTransport.obj
 0001:0000087b       _parseAllowedPeersInternal 1000187b f   socketTransport.obj
 0001:000009b1       _parseScopeId              100019b1 f   socketTransport.obj
 0001:000009f7       _readBooleanSysProp        100019f7 f   socketTransport.obj
 0001:00000a8e       _recv_fully                10001a8e f   socketTransport.obj
 0001:00000ac7       _send_fully                10001ac7 f   socketTransport.obj
 0001:00000b00       _setLastError              10001b00 f   socketTransport.obj
 0001:00000be3       _setOptionsCommon          10001be3 f   socketTransport.obj
 0001:00000c39       _socketTransport_accept@20 10001c39 f   socketTransport.obj
 0001:00000f6d       _socketTransport_attach@24 10001f6d f   socketTransport.obj
 0001:0000108c       _socketTransport_close@4   1000208c f   socketTransport.obj
 0001:000010c4       _socketTransport_getCapabilities@8 100020c4 f   socketTransport.obj
 0001:000010e9       _socketTransport_getLastError@8 100020e9 f   socketTransport.obj
 0001:00001132       _socketTransport_isOpen@4  10002132 f   socketTransport.obj
 0001:0000113f       _socketTransport_readPacket@8 1000213f f   socketTransport.obj
 0001:000012b8       _socketTransport_setConfiguration@8 100022b8 f   socketTransport.obj
 0001:0000134b       _socketTransport_startListening@12 1000234b f   socketTransport.obj
 0001:00001488       _socketTransport_stopListening@4 10002488 f   socketTransport.obj
 0001:000014cc       _socketTransport_writePacket@8 100024cc f   socketTransport.obj
 0001:00001669       _startListening            10002669 f   socketTransport.obj
 0001:00001f00       $$000000                   10002f00     MSVCRT:lldiv.obj
 0001:00001faa       ?dllmain_crt_dispatch@@YGHQAUHINSTANCE__@@KQAX@Z 10002faa f   MSVCRT:dll_dllmain.obj
 0001:00001ffd       ?dllmain_crt_process_attach@@YAHQAUHINSTANCE__@@QAX@Z 10002ffd f   MSVCRT:dll_dllmain.obj
 0001:00002104       ?dllmain_crt_process_detach@@YAH_N@Z 10003104 f   MSVCRT:dll_dllmain.obj
 0001:000021b4       ?dllmain_dispatch@@YAHQAUHINSTANCE__@@KQAX@Z 100031b4 f   MSVCRT:dll_dllmain.obj
 0001:000022bf       ?dllmain_raw@@YGHQAUHINSTANCE__@@KQAX@Z 100032bf f   MSVCRT:dll_dllmain.obj
 0001:0000230d       ___get_entropy             1000330d f   MSVCRT:gs_support.obj
 0001:000023e0       ?find_pe_section@@YAPAU_IMAGE_SECTION_HEADER@@QAEI@Z 100033e0 f   MSVCRT:utility.obj
 0001:00002840       $$000000                   10003840     MSVCRT:sehprolg4.obj
 0002:000006c0       _winsock_errors            100046c0     socket_md.obj
 0002:00000dd4       _GS_ExceptionPointers      10004dd4     MSVCRT:gs_report.obj
 0002:000011a8       __sehtable$?dllmain_crt_process_attach@@YAHQAUHINSTANCE__@@QAX@Z 100051a8     MSVCRT:dll_dllmain.obj
 0002:000011c8       __sehtable$?dllmain_crt_process_detach@@YAH_N@Z 100051c8     MSVCRT:dll_dllmain.obj
 0002:000011f0       __sehtable$?dllmain_dispatch@@YAHQAUHINSTANCE__@@KQAX@Z 100051f0     MSVCRT:dll_dllmain.obj
 0002:00001210       __sehtable$___scrt_is_nonwritable_in_current_image 10005210     MSVCRT:utility.obj
 0002:00001230       .edata                     10005230     dt_socket.exp
 0002:00001258       rgpv                       10005258     dt_socket.exp
 0002:0000125c       rgszName                   1000525c     dt_socket.exp
 0002:00001260       rgwOrd                     10005260     dt_socket.exp
 0002:00001262       szName                     10005262     dt_socket.exp
 0002:00001270       $N00001                    10005270     dt_socket.exp
 0002:000014b0       .idata$6                   100054b0     ws2_32:WS2_32.dll
 0002:000014ce       .idata$6                   100054ce     iphlpapi:IPHLPAPI.DLL
 0002:0000164c       .idata$6                   1000564c     kernel32:KERNEL32.dll
 0002:000016c6       .idata$6                   100056c6     vcruntime:VCRUNTIME140.dll
 0002:0000180a       .idata$6                   1000580a     ucrt:api-ms-win-crt-stdio-l1-1-0.dll
 0002:0000182a       .idata$6                   1000582a     ucrt:api-ms-win-crt-string-l1-1-0.dll
 0002:0000184c       .idata$6                   1000584c     ucrt:api-ms-win-crt-convert-l1-1-0.dll
 0002:0000186e       .idata$6                   1000586e     ucrt:api-ms-win-crt-runtime-l1-1-0.dll
 0003:00000000       _serverSocketFD            10006000     socketTransport.obj
 0003:00000004       _socketFD                  10006004     socketTransport.obj
 0003:00000008       _single_env                10006008     socketTransport.obj
 0003:0000000c       _preferredAddressFamily    1000600c     socketTransport.obj
 0003:00000038       _interface                 10006038     socketTransport.obj
 0003:00000068       _callback                  10006068     socketTransport.obj
 0003:0000006c       _jvm                       1000606c     socketTransport.obj
 0003:00000070       _tlsIndex                  10006070     socketTransport.obj
 0003:00000074       _initialized               10006074     socketTransport.obj
 0003:00000078       __peers                    10006078     socketTransport.obj
 0003:00000478       __peers_cnt                10006478     socketTransport.obj
 0003:0000047c       _allowOnlyIPv4             1000647c     socketTransport.obj
 0003:00000480       ?fileTime_1_1_70@?1??dbgsysCurrentTimeMillis@@9@9 10006480     socket_md.obj
 0003:00000488       _GS_ExceptionRecord        10006488     MSVCRT:gs_report.obj
 0003:000004d8       _GS_ContextRecord          100064d8     MSVCRT:gs_report.obj
 0003:000007a4       ?__proc_attached@@3HA      100067a4     MSVCRT:dll_dllmain.obj
 0003:000007c0       ?is_initialized_as_dll@@3_NA 100067c0     MSVCRT:utility.obj
 0003:000007c1       ?module_local_atexit_table_initialized@@3_NA 100067c1     MSVCRT:utility.obj
 0003:000007c4       ?module_local_atexit_table@@3U_onexit_table_t@@A 100067c4     MSVCRT:utility.obj
 0003:000007d0       ?module_local_at_quick_exit_table@@3U_onexit_table_t@@A 100067d0     MSVCRT:utility.obj
 0004:00000060       $R000000                   10007060     dt_socket.dll.res
